:1010000039C0000052C0000050C000004EC00000B7
:101010004CC000004AC0000048C0000046C00000AC
:1010200044C0000042C0000040C00000AAC300004D
:101030003CC000003AC0000038C0000036C00000CC
:1010400034C0000032C00000C6C100002EC0000045
:101050002CC000002AC0000028C0000026C00000EC
:1010600024C0000022C0000020C000001EC00000FC
:101070001CC0000011241FBECFEFD2E0DEBFCDBFE9
:1010800011E0A0E0B1E0EAE4FDE102C005900D92BC
:10109000A63DB107D9F721E0A6EDB1E001C01D9250
:1010A000A43FB207E1F72FD04EC6AACF8091D60158
:1010B000882341F18091E6019091E701A091E80138
:1010C000B091E90180784091DE015091DF0160919B
:1010D000E0017091E101481759076A077B0791F019
:1010E00025E0FA0120935700E89507B600FCFDCFF4
:1010F0008093DE019093DF01A093E001B093E101C2
:101100001092D601089584B7877F84BF88E10FB617
:10111000F89480936000109260000FBE90E080E829
:101120000FB6F89480936100909361000FBEC1E008
:10113000C5BF82E085BF16D3C0936F0083E0809364
:101140008100789411E043E0E42E01E054E0D52ED4
:1011500066E0C62E73E0B72EE2E0AE2E809100016D
:10116000882309F421C181E091E043D5F82E88233A
:1011700009F415C1C0E0D0E0FC1609F410C181E00B
:1011800091E053D59091D701992311F08A33D1F48E
:101190001092DD014091E2015091E3016091E40180
:1011A0007091E5014093E6015093E7016093E801F7
:1011B0007093E9011092DA018A3309F0EEC00093CE
:1011C000D701EBC02FEB280F263010F4875304C053
:1011D00080538A3008F0E1C04091D9014295407FA8
:1011E000482B4093D9018091DA0181278093DA015D
:1011F0008111D3C08091DD01963009F4BEC0840F07
:101200008093DD01933051F1F8F4913011F1923077
:1012100009F0C1C050E0542F44278091E60190911D
:10122000E701A091E801B091E901840F951FA11D8C
:10123000B11D8093E6019093E701A093E801B0937C
:10124000E901B092D701A9C09430F9F0953049F185
:10125000A2C04093DC01A092D7019FC08091E6011B
:101260009091E701A091E801B091E901840F911DEF
:10127000A11DB11D8093E6019093E701A093E801C1
:10128000B093E901D092D70188C04093DB018091EF
:10129000DC01882311F085E001C086E08093D7014E
:1012A0007CC02091DC0121502093DC018091E6017B
:1012B0009091E701A091E801B091E901811530E139
:1012C0009307A105B10528F01092D7011092D6011D
:1012D00064C020FF03C04093D8015FC050E0542F8A
:1012E00044272091D801422B2091DB01223039F193
:1012F000243079F121113AC02091D60121110CC07E
:10130000E091DE01F091DF01E0925700E89507B629
:1013100000FCFDCF0093D601FC010A011093570099
:10132000E89511240296A11DB11D8093E6019093CA
:10133000E701A093E801B093E901B8DE17C060E0CF
:1013400070E094E0440F551F661F771F9A95D1F700
:1013500005C060E070E0BA01552744274093E201E0
:101360005093E3016093E4017093E5018091DC0107
:10137000811113C0C092D70110C050E0819590E058
:101380004817590751F492DE8091DB01813029F42E
:101390001092000102C01092D7012196EDCE81E09B
:1013A00091E0DAD383D3DACE8091E000816080933C
:1013B000E00082E49CED9093F5018093F4012CE031
:1013C00088E190E00FB6F894A895809360000FBE76
:1013D00020936000FFCF1F920F920FB60F9211243F
:1013E0000F900FBE0F901F9018950895089581E0FB
:1013F00091E077D31092D701089581E091E03AC44B
:10140000292F33272230310559F02330310569F077
:1014100021303105D9F482E190E029E831E01AC0A9
:1014200080E290E029E631E015C0992783309105EC
:1014300068F4FC01EE0FFF1FED5EFE4F208131814D
:10144000FC01E05FFE4F808190E004C080E090E00E
:1014500020E030E0FA0131832083089507B600FCD4
:10146000FDCFF999FECF23E0FB0120935700E895CB
:1014700007B600FCFDCF81E180935700E895089501
:1014800007B600FCFDCFF999FECF25E0FB012093C4
:101490005700E89507B600FCFDCF81E18093570027
:1014A000E895089507B600FCFDCFF999FECF21E03D
:1014B000FB010A0120935700E8951124089521E2C9
:1014C000FC01209357008491089529E0FC012093AA
:1014D000570084910895E1E0F0E089E0809357009F
:1014E0008491089507B600FCFDCFF999FECF809551
:1014F00099E0E1E0F0E0082E90935700E895089518
:101500002091F2013091F3012617370748F0611559
:10151000710539F42091E8002E772093E80001C08E
:10152000B90120E061157105C9F13EB3332309F417
:1015300042C0353009F441C03091E80033FD3FC06E
:101540003091E80032FF06C08091E80082FF29C098
:1015500080E008953091E80030FFE4CF2091F20060
:1015600030E0FC01281B390BCF01820F931F61155E
:10157000710549F08830910530F481918093F10034
:1015800061507109F1CF21E0089709F020E08091C6
:10159000E8008E778093E800CF01C4CF2111C5CF3A
:1015A000D3CF8EB3882339F0853039F08091E800AD
:1015B00083FFCACF04C082E0089583E0089581E0EC
:1015C00008958F708093E900EBEEF0E080818160F8
:1015D0008083EDEEF0E010826093EC004083809118
:1015E000EE00881F8827881F08950F931F93CF93BD
:1015F000DF93062FEC0110E0101769F19881992311
:1016000039F12C81E981FA816B81892F8F708530C6
:1016100010F080E021C0223010F056E001C052E00E
:1016200028E030E040E02E173F0720F44F5F220F04
:10163000331FF9CF4295407F452B991F9927991F5A
:101640006295660F660F607C692BBBDF882309F308
:101650001F5F2596D1CF81E0DF91CF911F910F9130
:1016600008958091EC0187FD05C08091E80080FF1E
:101670000DC010C08091E80082FD04C08EB38111BE
:10168000F9CF08958091E8008B7707C08EB3811160
:10169000ECCF08958091E8008E778093E80008955C
:1016A0008091E4009091E50045E62091EC0020FF58
:1016B00020C02091E80020FD20C02EB3222389F015
:1016C000253089F02091EB0025FD0FC02091E4002A
:1016D0003091E5002817390741F3415041F0C90125
:1016E000E4CF82E0089583E0089581E0089584E0E6
:1016F00008952091E80022FFE0CF80E008953BD0DC
:101700003DD08091D8008F778093D8008091D80009
:1017100080688093D8008091D8008F7D8093D80016
:1017200019BC82E089BD09B400FEFDCF1EBA10923B
:10173000EA0142E060E080E044DF8091E1008E7FDA
:101740008093E1008091E20081608093E2008091CB
:10175000E20088608093E2008091E0008E7F8093B9
:10176000E0000895E3E6F0E080818E7F808381E0F1
:101770008093EB01C4CF1092E20008951092E10033
:1017800008951F920F920FB60F9211242F933F933B
:101790004F935F936F937F938F939F93AF93BF9379
:1017A000EF93FF938091E10080FF16C08091E200EB
:1017B00080FF12C08091E2008E7F8093E2008091D2
:1017C000E20080618093E2008091D8008062809383
:1017D000D80019BC1EBA0ADE8091E10084FF2DC03A
:1017E0008091E20084FF29C019BC82E089BD09B460
:1017F00000FEFDCF8091D8008F7D8093D80080912E
:10180000E1008F7E8093E1008091E2008F7E8093E3
:10181000E2008091E20081608093E2008091EA0121
:10182000882311F084E007C08091E30087FF02C0A5
:1018300083E001C081E08EBBD8DD8091E10083FFB1
:1018400021C08091E20083FF1DC08091E100877F6D
:101850008093E10082E08EBB1092EA018091E1006A
:101860008E7F8093E1008091E2008E7F8093E20082
:101870008091E20080618093E20042E060E080E0DD
:10188000A0DE13D1FF91EF91BF91AF919F918F9106
:101890007F916F915F914F913F912F910F900FBE6C
:1018A0000F901F9018951F93CF93DF9300D0CDB763
:1018B000DEB7ECEEF1E08091F100819381E0E43F4E
:1018C000F807C9F79ADD8091E80083FFDAC09091AC
:1018D000EC018091ED01853009F465C030F4813070
:1018E00059F168F0833041F1CCC0883009F49CC0D4
:1018F000893009F4ABC0863009F0C3C075C0903898
:1019000081F0923809F0BDC08091F0018F70809312
:10191000E9009091EB0095FB992790F91092E9006E
:1019200001C090E08091E800877F8093E800909369
:10193000F1001092F10083C0292F2D7F09F0A1C082
:10194000923009F09EC09091EE01911126C0209135
:10195000F0012F7009F495C02093E9009091EB00FD
:1019600090FF1BC0833021F48091EB00806213C094
:101970008091EB0080618093EB0081E090E0022E8B
:1019800001C0880F0A94EAF78093EA001092EA00F7
:101990008091EB0088608093EB001092E9008091C9
:1019A000E800877F4FC091116CC01091EE011F7746
:1019B0008091E3008078812B8093E3008091E800A0
:1019C000877F8093E8004DDE8091E80080FFFCCFA8
:1019D0008091E30080688093E300112311F083E09D
:1019E00001C082E08EBB4DC09058923008F049C0D3
:1019F000AE014F5F5F4F6091F0018091EE019091D9
:101A0000EF01FEDC009709F43CC02091E800277F3D
:101A10002093E800BC0189819A8172DD8091E80001
:101A20008B778093E8002DC0903859F58091E800BD
:101A3000877F8093E8008091EA018093F100809194
:101A4000E8008E778093E8000CDE1BC0911119C06E
:101A50009091EE019230A8F48091E800877F809306
:101A6000E8009093EA01FDDD8091EA01811104C054
:101A70008091E30087FF02C084E001C081E08EBB5B
:101A8000B6DC8091E80083FF0AC08091E800877F80
:101A90008093E8008091EB0080628093EB000F90D0
:101AA0000F90DF91CF911F9108950895CF938EB33A
:101AB0008823A9F08091E9008F709091EC0090FF4D
:101AC00002C090E801C090E0C92FC82B1092E90035
:101AD0008091E80083FDE7DECF70C093E900CF91ED
:101AE0000895CF93DF93EC011E861D8688E18D87D4
:101AF00082E08C83898761E0CE01019676DD8823C0
:101B000031F061E0CE010696DF91CF916ECD80E09D
:101B1000DF91CF9108952EB32430E1F4FC0181814F
:101B20008F708093E9008091F200882389F0909172
:101B3000E8008091E8008E778093E80095FD08C06A
:101B4000AFDD811108C08091E8008E778093E800B6
:101B500080E0089582E00895CF93DF93EC018EB387
:101B6000843009F043C089818F708093E9008091AF
:101B7000E80080FF02C0CE01CEDF8E858823B1F160
:101B80002E812F7081E090E0AC0102C0440F551F00
:101B90002A95E2F74093EA001092EA0029812F701B
:101BA000022E01C0880F0A94EAF78093EA0010928F
:101BB000EA008E818F708093E9008091EB00806154
:101BC0008093EB008091EB0088608093EB0089812B
:101BD0008F708093E9008091EB0080618093EB002F
:101BE0008091EB0088608093EB001E86DF91CF919F
:101BF00008952EB3243091F4FC0186818F70809378
:101C0000E9008091E80082FF09C08091F200811113
:101C100008C08091E8008B778093E80080E090E036
:101C200008958091F20090E008952EB3243019F0C9
:101C30008FEF9FEF0895FC0186818F708093E900FC
:101C40008091E80082FFF4CF8091F200882321F098
:101C50002091F10030E002C02FEF3FEF8091F200C1
:101C6000811105C08091E8008B778093E800C9015D
:101C700008950895CF93DF93EC018091E80083FFEE
:101C80005FC0888190E02091F0013091F101281728
:101C9000390709F055C08091ED01813051F120F0F4
:101CA000823009F43DC04CC08091EC01813A09F0CA
:101CB00047C08091E800877F8093E8008091E8002A
:101CC00080FD04C08EB38111F9CF3AC0EB85FC854D
:101CD000DF010D900020E9F7BD01615071096E1B15
:101CE0007F0B7093F1006093F1008B859C8508DC7D
:101CF00014C08091EC01813A19F58091E800877F4A
:101D00008093E8008091E80080FD04C08EB38111CB
:101D1000F9CF16C08D858093F100DF91CF91A1CCD2
:101D20008091EC01813261F48091E800877F80939B
:101D3000E80097DC81E08E87CE01DF91CF9199CFCB
:0A1D4000DF91CF910895F894FFCFD2
:101D4A000100834000000104400000019B010000E3
:101D5A0004183065014B01190130034C0055004647
:101D6A0000410020005000720069006E0074006596
:101D7A00007200200042006F006F0074006C006F58
:101D8A0000610064006500720000001803440065E9
:101D9A000061006E002000430061006D0065007262
:101DAA000061000000040309040902200001010087
:101DBA00803209040000020701020007058302407D
:101DCA000005070504024000051201100100000089
:101DDA0008EB036B200100010200014D46473A4718
:101DEA00656E657269633B4D444C3A47656E657230
:101DFA0069635F2F5F546578745F4F6E6C793B43FC
:101E0A004D443A313238342E343B434C533A5052D3
:061E1A00494E5445520040
:101FA0005DCA6ECA7FCA8BCA90CA95CA9BCA089579
:081FB0000895089508950895B5
:101FE000DFCFDFCFDFCFDFCFDFCFDFCFDFCFDFCF81
:081FF000DFCFDFCFDFCFDFCF31
:081FF8000010000020DFFBDCFB
:0400000300001000E9
:00000001FF
